:020000040000FA
:020000000A28CC
:0800080010308B000000903065
:100010008B00090083160130860083128601903020
:100020008B000A309200323086009E2006184B2842
:10003000543086009E2006184B28983086009E205B
:1000400006184B28543086009E2006184B28323064
:1000500086009E2006184B28103086009E20061829
:100060004B28FE3086009E2006184B2886019E20D5
:1000700006184B28920B1328A520FE308600A520D9
:100080008601A520FE308600A5208601A5200B1143
:10009000630000000A28860106184B28612093009F
:1000A0008600A5208601A52013088600A5208601CC
:1000B000A52013088600A520A5208601A520A5203F
:1000C0001328BA30860097200618BA3400000000C2
:1000D0001030860097200618103400000000AA3067
:1000E000860097200618AA340000000022308600FF
:1000F0009720061822340000000032308600972036
:100100000618323400000000EE30860097200618F2
:10011000EE3461283E308D0000008D0B8C280800E5
:1001200064308E0000008A208E0B92280800053073
:100130008F00000090208F0B99280800323090002B
:1001400000009020900BA02808006430910000006F
:080150009020910BA728080084
:02400E00F23F7F
:00000001FF
